:100000000C94B7040C94FF040C94FF040C94FF04AC
:100010000C94FF040C94FF040C94FF040C94FF0454
:100020000C94FF040C94FF040C94FF040C941A1D10
:100030000C94FF040C94F11C0C94FF040C94FF042A
:100040000C94FF040C94FF040C94FF040C94CB1C40
:100050000C94FF040C94FF040C94FF040C94FF0414
:100060000C94FF040C94FF040C94FF040C94FF0404
:100070000C94FF040631FF0974A1010975150026CF
:10008000FF009520750881020976150026FF00956E
:100090002075089102C005010902A1010901A10012
:1000A0008501050919012908150025019508750123
:1000B00081020501093009311581257F95027508F6
:1000C000810609381581257F950175088106050C83
:1000D0000A38021581257F950175088106C0C00583
:1000E000010980A10185021601002637001A81004E
:1000F0002AB700751095018100C0050C0901A10106
:100100008503160100269C021A01002A9C02751024
:1001100095018100C005010906A101050719E02923
:10012000E715002501950875018102950175088183
:1001300001050819012905950575019102950175BB
:100140000391010507190029FF150026FF009506F8
:1001500075088100C02831290A002832290A0028A0
:1001600033290A002834290A005D0A002530325854
:10017000005B006D6F64656C3A20253032580A00D0
:100180000A0025303258006D303131305F73656EB2
:1001900064206572723A20000A0025303258006DE2
:1001A000303131305F72656376206572723A2000BB
:1001B0002000253032580025583A25303862257302
:1001C0000A000A202030313233343536370A004CE9
:1001D00045443A20253032580A000A4C6F6F70208F
:1001E00073746172742E0A000A55534220636F6E55
:1001F000666967757265642E0A000A544D4B3A327F
:1002000064643934382F4C5546413A64366137645A
:10021000660A0009025400030100A032090400002C
:10022000010301010009211101000122400007051D
:10023000810308000A0904010001030102000921E9
:1002400011010001227F0007058203080001090453
:100250000200010300000009211101000122220017
:10026000070583032000011201100100000008EDC2
:10027000FE100101010102000132034D0030003186
:10028000003100300020006B006500790062006FD3
:1002900000610072006400200063006F006E007651
:1002A000006500720074006500720000000E0374A7
:1002B000002E006D002E006B002E000000040309CC
:1002C0000473797374656D3A20253034580A0063DD
:1002D0006F6E73756D65723A20253034580A003F91
:1002E000004D3E2000433E20000A00257500363AAE
:1002F00020776865656C5F74696D655F746F5F6DAD
:1003000061783A20000A00257500353A2077686543
:10031000656C5F6D61785F73706565643A20000A93
:1003200000257500343A2074696D655F746F5F6DE8
:1003300061783A20000A00257500333A206D617813
:100340005F73706565643A20000A00257500323AD3
:1003500020696E74657276616C286D73293A20008D
:100360000A00257500313A2064656C6179282A31CC
:10037000306D73293A20000A092D2056616C75658D
:1003800073202D0A004D3E004D25643E20003F00A5
:100390007365742064656661756C740A00433E2061
:1003A000000A002530325820006B6579626F617257
:1003B000643A2000041607090B0A1D1B0619640580
:1003C000141A08151C171E1F202123222E26242D47
:1003D00025273012182F0C13280F0D340E33313609
:1003E000381110372B2C352A7F80807B79397A8021
:1003F0008080808080634F808080505351808080D7
:1004000058525780808062595A5B5C5D5E5F8060A5
:10041000618080808080568080806680548080806B
:1004200080558080290A002575002F002575005D04
:100430002800256400200025640020002564002099
:10044000002564007C0025303258006D6F7573659F
:100450006B6579205B62746E7C78207920762068E9
:100460005D287265702F61636C293A205B000A0970
:100470002D204D61676963202D0A643A0964656225
:1004800075670A783A096465627567206D617472F0
:1004900069780A6B3A096465627567206B657962F1
:1004A0006F6172640A6D3A096465627567206D6FE9
:1004B0007573650A763A0976657273696F6E0A73A9
:1004C0003A097374617475730A633A09636F6E73E2
:1004D0006F6C65206D6F64650A302D343A096C616C
:1004E000796572302D34284631302D4634290A5032
:1004F0006175733A09626F6F746C6F616465720A3B
:10050000000A092D20436F6E736F6C65202D0A451C
:1005100053432F713A09717569740A6D3A096D6F09
:100520007573656B65790A003F0074696D65725F6C
:1005300072656164333228293A202530346C580AB8
:10054000006B6579626F6172645F69646C653A2003
:1005500025580A006B6579626F6172645F70726F13
:10056000746F636F6C3A2025580A00686F73745F6C
:100570006B6579626F6172645F6C65647328293A98
:100580002025580A000A092D2053746174757320C0
:100590002D0A004743433A20372E332E3020415650
:1005A000522D4C4942433A20322E302E30204156B3
:1005B000525F415243483A2061767233350A004F08
:1005C0005054494F4E533A204C554641204D4F55BB
:1005D00053454B45592045585452414B45592043AA
:1005E0004F4E534F4C4520434F4D4D414E44204BB1
:1005F00045594D41505F53454354494F4E20343087
:1006000039360A004255494C443A20326464393440
:1006100038202831323A30333A3538204A616E205A
:1006200033302032303233290A005649443A2030E0
:10063000784645454428742E6D2E6B2E292050494E
:10064000443A20307830313130284D30313130204B
:100650006B6579626F61726420636F6E7665727428
:10066000657229205645523A203078303130310AAF
:1006700000444553433A20636F6E76657274204D93
:1006800030313130206B6579626F61726420746F34
:10069000205553420A000A092D2056657273696F6E
:1006A0006E202D0A000A6D6F7573653A206F6666BD
:1006B0000A000A6D6F7573653A206F6E0A000A6B47
:1006C0006579626F6172643A206F66660A000A6B30
:1006D0006579626F6172643A206F6E0A000A6D611B
:1006E000747269783A206F66660A000A6D617472E6
:1006F00069783A206F6E0A000A64656275673A206D
:100700006F6E0A000A64656275673A206F66660A52
:10071000000A0A626F6F746C6F616465722E2E2E10
:100720002000433E20006D6B5F776865656C5F74E9
:10073000696D655F746F5F6D6178203D2025640A87
:10074000006D6B5F776865656C5F6D61785F737076
:10075000656564203D2025640A006D6B5F74696DDA
:10076000655F746F5F6D6178203D2025640A006DC0
:100770006B5F6D61785F7370656564203D202564F3
:100780000A006D6B5F696E74657276616C203D2046
:1007900025640A006D6B5F64656C6179203D2025DE
:1007A000640A006D6B5F776865656C5F74696D6581
:1007B0005F746F5F6D6178203D2025640A006D6B6A
:1007C0005F776865656C5F6D61785F7370656564A0
:1007D000203D2025640A006D6B5F74696D655F7450
:1007E0006F5F6D6178203D2025640A006D6B5F6D41
:1007F00061785F7370656564203D2025640A006D33
:100800006B5F696E74657276616C203D2025640AA9
:10081000006D6B5F64656C6179203D2025640A0082
:1008200077686572652064656C74613A20637572DF
:10083000736F723D25642C20776865656C3D256477
:100840000A53656520687474703A2F2F656E2E7791
:10085000696B6970656469612E6F72672F77696B68
:10086000692F4D6F7573655F6B6579730A000A09AF
:100870002D204D6F7573656B6579202D0A455343A7
:100880002F713A09717569740A313A0964656C61AE
:1008900079282A31306D73290A323A09696E7465F4
:1008A0007276616C286D73290A333A096D61785F3D
:1008B00073706565640A343A0974696D655F746FB5
:1008C0005F6D61780A353A09776865656C5F6D61BF
:1008D000785F73706565640A363A09776865656C98
:1008E0005F74696D655F746F5F6D61780A0A703A55
:1008F000097072696E742076616C7565730A643A6A
:10090000097365742064656661756C74730A75702B
:100910003A092B310A646F776E3A092D310A7067F4
:1009200075703A092B31300A7067646F776E3A0937
:100930002D31300A0A7370656564203D2064656C52
:100940007461202A206D61785F7370656564202A68
:100950002028726570656174202F2074696D655F51
:10096000746F5F6D6178290A004C25640A001124B8
:100970001FBECFEFD4E0DEBFCDBF04B603FE28C05C
:100980008091460390914703A0914803B091490399
:100990008730904BA740B04BD9F410924603109289
:1009A0004703109248031092490314BE0FB6F894FF
:1009B000A89580916000886180936000109260002B
:1009C0000FBE1092010810920008E0E0F8E30995CC
:1009D00011E0A0E0B1E0E4E6F4E402C005900D927D
:1009E000A433B107D9F723E0A4E3B1E001C01D921D
:1009F000A634B207E1F70E94CB1D0C9430220C9470
:100A00000000FF93EF93E0913401F09135013097AE
:100A100009F00995EF91FF910895FC0185918030CF
:100A200011F0EFDFFBCF0895FF27E0E230E247FF50
:100A30000CC0419597FF09C0EDE2609570958095D7
:100A40009095611D711D811D911D27FF02C021958B
:100A500030E350E2AA27660F771F881F991FAA1F4D
:100A6000A41710F0A41B63955A95A9F7AA3008F0B3
:100A7000A95FA05DAF93F39561157105810591059F
:100A800041F7ED3211F4EF93F395F21718F43F9319
:100A9000F395FBCF8F91B5DFFA95E1F70895E991D2
:100AA000F9918591803021F0853219F0AADFF9CFD4
:100AB000089520E0E89455915532C1F3503311F474
:100AC000689455915A3348F4505390F3220F022EF4
:100AD000220F220F200D250FF4CF0EF421958991BE
:100AE0009991533619F3533729F1533559F1BC0114
:100AF00088279927E8945C3621F489919991689424
:100B00005591543639F446EF7EF077FF0DC08FEFE4
:100B10009FEF0AC055374AE039F0583540E121F0DF
:100B2000523642E009F00895FF93EF937DDFEF9195
:100B3000FF91B7CFFF93EF93FC0181918030B9F320
:100B400060DFFBCFFF93EF9368DFF1CFDF93CF93AD
:100B5000CDB7DEB72596A3DFCF91DF9108958091C1
:100B6000300380FF0CC06091140170E075956795AB
:100B7000759567956115710559F1862F089581FF67
:100B800006C06091140170E075956795F3CF609190
:100B9000140170E082FD0CC0609131036623A9F05E
:100BA000209113018091140190E0621730F0BC0194
:100BB00060387105F8F28FE7089570E00E94F12126
:100BC000622F70E00E940222F3CF61E070E0D5CF87
:100BD00081E008958091300380FF11C0809116015B
:100BE00090E065E070E00E94F121959587959595DC
:100BF000879580389105B0F50097B1F1089581FF90
:100C00000AC08091160190E065E070E00E94F12139
:100C100095958795EECF82FF08C08091160190E0F0
:100C200065E070E00E94F121E4CF3091310333237D
:100C3000B1F0209115018091160190E065E070E01F
:100C40000E94F121BC013217A0F6832F90E00E9490
:100C5000F121622F70E00E940222CB01CACF85E011
:100C600090E008958FE7089581E00895E72FF0E080
:100C700093E0EE0FFF1F9A95E1F7E60FF11DEC549C
:100C8000FC4F6491E62FE295E77090E023E0880F37
:100C9000991F2A95E1F78E0F911D34E0880F991F57
:100CA0003A95E1F7E62FEF70E80FF92FF11DEE0FFF
:100CB000FF1FE050F8498591949108952FB7F8945B
:100CC00080913B0390913C03A0913D03B0913E0382
:100CD0002FBF0895E6E3F2E09281891301C01282EA
:100CE000319692E0EC33F907B9F70895A8E3B2E042
:100CF000EFEF90E02D91821751F0EF3F19F42111A1
:100D000001C0E92F9F5F9630A9F7EF3F09F40895DE
:100D10000E2E000CFF0BEA5CFD4F828308954F926C
:100D20005F926F927F929F92AF92BF92CF92DF922B
:100D3000EF92FF920F931F93CF93DF9300D000D0D9
:100D40001F92CDB7DEB76B837C838D837A018C8154
:100D50009D81892B49F08FEFF81204C081E09FEF4D
:100D6000491719F080E001C081E080FD6AC00F2DB5
:100D700010E0CE2CD12C8B81882309F456C04090F2
:100D8000B8025090B9026090BA027090BB02809194
:100D9000420390914303A0914403B0914503482A34
:100DA000592A6A2A7B2A2FE1A22EB12C9A2CD30130
:100DB000C2010A2C04C0B695A795979587950A9409
:100DC000D2F780FD2BC081E0A81AB10878F7912CEA
:100DD000F80193E0EE0FFF1F9A95E1F7E454FD4F01
:100DE000EC0DFD1D9082E982FA8269817A81892D5C
:100DF0000F900F900F900F900F90DF91CF911F9158
:100E00000F91FF90EF90DF90CF90BF90AF909F90A9
:100E10007F906F905F904F900C943606B7018A2DAB
:100E20000E943606019779F2D3CFF80183E0EE0FE6
:100E3000FF1F8A95E1F7E454FD4FEC0DFD1D9080F6
:100E4000D2CF90E080E00F900F900F900F900F9016
:100E5000DF91CF911F910F91FF90EF90DF90CF9096
:100E6000BF90AF909F907F906F905F904F9008954C
:100E700041E050E060E070E004C0440F551F661F81
:100E8000771F8A95D2F7409550956095709580911F
:100E9000B8029091B902A091BA02B091BB0284232A
:100EA0009523A623B7238093B8029093B902A09309
:100EB000BA02B093BB02089541E050E060E070E0F8
:100EC00004C0440F551F661F771F8A95D2F7809183
:100ED000B8029091B902A091BA02B091BB02842BE2
:100EE000952BA62BB72B8093B8029093B902A093B1
:100EF000BA02B093BB0208958091B7029091860226
:100F0000981301C008958F5F8770FACF1F93CF9316
:100F1000DF9300D000D01F92CDB7DEB7942F498366
:100F2000252F5A836B837C838D834C815D8181E087
:100F3000452B31F02F3F19F481E09F3F09F080E00D
:100F4000182F117080FD2CC049815A816B817C81E2
:100F50008D810E948F06292F22952F702C3078F4D6
:100F60002A30A8F422502230C8F0812F0F900F9021
:100F70000F900F900F90DF91CF911F9108952C301B
:100F800011F02F3091F793FB112710F9EECF803C31
:100F900028F0803E50F3815F833038F311E0E5CFD5
:100FA00010E0E3CFE0913203F0913303309721F06A
:100FB0000190F081E02D099480E008951092E20004
:100FC0001092E100E0EEF0E0808181608083E8ED46
:100FD000F0E080818F77808319BCE3E6F0E08081C8
:100FE000816080831092640208950E94DE07F89465
:100FF00087E797E7909301088093000887E090EBDC
:10100000DC018093460390934703A0934803B09379
:10101000490388E19CE00FB6F894A895809360009E
:101020000FBE90936000FFCFFC01809178029091F9
:10103000790286179707A0F06115710529F4909140
:10104000E8009E779093E80090E06115710551F4F7
:10105000911108C08091E80082FF32C080E00895BD
:10106000BC01F2CF80917A028823B1F18530B1F1D1
:101070008091E80083FD2EC08091E80082FDEACFD8
:101080008091E80080FFE1CF2091F20030E061150F
:10109000710519F02830310558F091E028303105FC
:1010A00009F090E02091E8002E772093E800CDCF62
:1010B00081918093F100615071092F5F3F4FE7CF1D
:1010C00080917A02882341F0853041F08091E800D8
:1010D00083FFC0CF81E0089582E0089583E0089502
:1010E0002091E4003091E50085E69091EC0090FFBE
:1010F00006C09091E80090FF06C080E008959091AE
:10110000E80092FDFACF90917A02992391F0953000
:1011100091F09091EB0095FD10C04091E40050914A
:10112000E5002417350709F381509A01F1F684E0B0
:10113000089582E0089583E0089581E00895809104
:10114000720287FF13C08091E80082FF06C0809181
:10115000E8008B778093E80004C080917A028111C7
:10116000F2CF089580917A028823D9F38091E80024
:1011700080FFF8CF8091E8008E77ECCF982F909386
:10118000E900242F762F50E0891731F07091EC00A0
:101190002091ED005091F00021FD07C09F5F953038
:1011A00071F78093E90081E008953091EB003E7F74
:1011B0003093EB003091ED003D7F3093ED003091A6
:1011C000EB0031603093EB007093EC002093ED0066
:1011D0005093F0002091EE0027FDE0CF80E00895CD
:1011E00080916602089580914202811113C09FB7D9
:1011F000F89440913B0350913C0360913D03709102
:101200003E039FBF443C59406105710518F081E0E1
:10121000809342020895EF92FF920F931F93CF9312
:10122000DF93D82F0FB607FE46C080917A02843034
:1012300079F08091040190E001962091060130E060
:1012400082239323209105012817190609F0C9C0AC
:101250000E94F30881110FC08091040190E0019673
:101260002091060130E08223932320910501281765
:10127000190609F0B6C00E945E068C01C091E90013
:10128000CF708091EC0080FD37C080E0C82B83E0F8
:101290008093E90085E0E82E8091EB0085FD08C091
:1012A0008091EB0080FF04C08091EE0087FD44C078
:1012B000CF70C093E900E09104018E2F90E0019679
:1012C0002091060130E08223932320910501281705
:1012D000190609F47EC08091020190910301E80F84
:1012E000F92FF11DD083809104018F5F9091060149
:1012F0008923809304016DC080E8C8CFE09102018A
:10130000F0910301E80FF11D90818F5F209106019C
:101310008223809305019093F1008091E80085FD80
:101320000BC08091E80080FF07C08091E8008E77B5
:101330008093E800E0920101809105019091040101
:10134000981741F19091E80095FDD8CF80E029C031
:101350001092F1002EC08091040190E0019620913E
:10136000060130E0822393232091050128171906F6
:1013700009F09ECFF0900101FF2009F499CF0E945F
:101380005E068017910709F487CFFA94F092010165
:101390008C0182CF8091E80085FFD8CFD093F100F7
:1013A00081E09091F200992379F09091E80090FF0C
:1013B0000BC09091E80095FDCBCF9091E8009E770F
:1013C0009093E800E0920101882329F2CF70C09346
:1013D000E90080E0DF91CF911F910F91FF90EF9096
:1013E0000895E091040177CF5098589A089558983D
:1013F000509A08955198599A08958B3749F08F3F24
:1014000039F0282F30E0359527952F738078822B7F
:1014100008958330C9F128F4813061F0823019F1E8
:101420000895853009F452C008F43FC0863009F4AD
:101430005EC0089580911801681790F4861B809310
:101440001801809118011F928F9381E198E09F937A
:101450008F930E94A6050F900F900F900F90089504
:1014600010921801EECF80911701681750F4861B77
:1014700080931701809117011F928F938FEF97E050
:10148000E6CF10921701F6CF80911601681750F43D
:10149000861B80931601809116011F928F938CEE0C
:1014A00097E0D5CF10921601F6CF809115016817FD
:1014B00050F4861B80931501809115011F928F9324
:1014C00087ED97E0C4CF10921501F6CF80911401FB
:1014D000681750F4861B80931401809114011F92A9
:1014E0008F938EEB97E0B3CF10921401F6CF8091DB
:1014F0001301681750F4861B809313018091130128
:101500001F928F9383EA97E0A2CF10921301F6CF38
:10151000833009F445C028F4813061F0823049F10C
:101520000895853009F46AC008F451C0863009F482
:101530007CC0089580911801482F460F5527551FEC
:101540004F3F510594F4680F609318018091180182
:101550001F928F9384E997E09F938F930E94A60533
:101560000F900F900F900F9008958FEF80931801B8
:10157000EDCF80911701482F460F5527551F4F3F3C
:10158000510554F4680F60931701809117011F9261
:101590008F9382E897E0E0CF8FEF80931701F5CF2C
:1015A00080911601482F460F5527551F4F3F510573
:1015B00054F4680F60931601809116011F928F9367
:1015C0008FE697E0C9CF8FEF80931601F5CF80911A
:1015D0001501482F460F5527551F4F3F510554F40D
:1015E000680F60931501809115011F928F938AE512
:1015F00097E0B2CF8FEF80931501F5CF8091140162
:10160000482F460F5527551F4F3F510554F4680F7B
:1016100060931401809114011F928F9381E497E0ED
:101620009BCF8FEF80931401F5CF80911301482F4A
:10163000460F5527551F4F3F510554F4680F6093CF
:101640001301809113011F928F9386E297E084CF5C
:101650008FEF80931301F5CFCF93DF9320917D021D
:1016600030917E022817390701F190937E02809312
:101670007D02E0913203F09133033097B1F0EC0139
:101680000084F185E02D09958091410385708530B6
:1016900061F4DF93CF938FEC92E09F938F930E943E
:1016A000A6050F900F900F900F90DF91CF910895A6
:1016B000CF93DF9320917B0230917C02281739076A
:1016C00001F190937C0280937B02E0913203F091D0
:1016D00033033097B1F0EC010680F781E02D0995D6
:1016E000809141038570853061F4DF93CF9381EC65
:1016F00092E09F938F930E94A6050F900F900F90FA
:101700000F90DF91CF9108958EE698E00E940D052D
:101710001F9281E08F931F9285E08F9380E298E083
:101720009F938F930E94A6050F900F900F900F909C
:101730000F900F900895CF938091410383FF7EC057
:101740008BE494E00E940D05809136031F928F93E5
:1017500086E494E09F938F930E94A60584E494E02E
:101760000E940D0580913703282F082E000C330BA3
:101770003F938F9381E494E09F938F930E94A605FB
:101780008FE394E00E940D0580913803282F082EE6
:10179000000C330B3F938F938CE394E09F938F93D4
:1017A0000E94A6058AE394E00E940D05809139030A
:1017B000282F082E000C330B3F938F9387E394E080
:1017C0009F938F930E94A60585E394E00E940D05E8
:1017D00080913A03282F082E000C330B3F938F93F0
:1017E00082E394E09F938F930E94A6058FE294E09A
:1017F0000E940D05809131031F928F938CE294E03B
:101800009F938F930E94A6058AE294E00E940D05A3
:10181000809130031F928F9387E294E09F938F9380
:101820000E94A60584E294E00E940D058DB79EB744
:101830004C960FB6F8949EBF0FBE8DBFE091320359
:10184000F0913303309751F0C09136030480F58155
:10185000E02D86E393E00995C09336030E945E066F
:101860009093350380933403CF9108950F931F9382
:10187000CF93DF9380912E0390912D03892B80933A
:10188000360290912C03992389F0892B809336029C
:10189000E7E3F2E02EE332E080E0919191118F5F77
:1018A0002E173F07D1F7811110922C03E0913203DC
:1018B000F09133033097B1F10280F381E02D86E39C
:1018C00092E009958091410382FF2CC080FF04C003
:1018D00089EA93E00E940D05D0E0C0E003EA13E03E
:1018E0008091410380FF0EC0FE01EA5CFD4F8081C4
:1018F0001F928F931F930F930E94A6050F900F9036
:101900000F900F902196C830D10551F78091410377
:1019100080FF08C081EA93E0DF91CF911F910F9182
:101920000C940D05DF91CF911F910F9108951092A6
:101930002E0310922D03E6E3F2E01182128213824D
:1019400014821582168217820E94360C85E0E6E327
:10195000F3E0DF011D928A95E9F7109231031092AE
:1019600030030E949B0B90E080E00E94580B90E0B7
:1019700080E00C942C0BCF93C82F1F928F9389E695
:1019800099E09F938F930E94A60581E090E0A0E0EC
:10199000B0E004C0880F991FAA1FBB1FCA95D2F7D9
:1019A0008093420390934303A0934403B093450371
:1019B0000F900F900F900F90CF910C94970C0F9366
:1019C0001F93CF93DF93CDB7DEB7AA970FB6F894E6
:1019D000DEBF0FBECDBF80917A02882309F452C1C9
:1019E0001091E9001F708091EC0080FF39C080E801
:1019F000182B1092E9008091E80083FF40C1E2E7D4
:101A0000F2E08AE792E02091F10021938E179F0780
:101A1000D1F780917302833009F470C018F58130DA
:101A200009F447C0823009F4DEC08091E80083FFEA
:101A300018C180917202909173029A3008F011C11E
:101A4000E92FF0E0EA5DF24F0C941622040E2A0E04
:101A5000310E2A0E310E8C0EAE0E310EA90FB60FBE
:101A600080E0C6CF8A3009F4ADC08B3009F47DC068
:101A70008930D9F6809172028132B9F6809176026E
:101A800090917702892B89F68091E800877F809377
:101A9000E8008091E80082FF2CC08091F1008093E3
:101AA00066028091E8008B778093E8000E949F088F
:101AB000BCCF80917202813A09F0B7CF8091E800E3
:101AC000877F8093E8008091760290917702892B3E
:101AD00061F060E090E080E070E00E941408809186
:101AE000E8008B778093E800A0CF68E087E692E07B
:101AF000F3CF80917A028111CCCF97CF809172027F
:101B0000813A09F092CF8091760290917702892BE9
:101B1000A1F48091E800877F8093E8008091E8003D
:101B200080FFFCCF809112018093F1008091E8004A
:101B30008E778093E8000E949F08809176029091B2
:101B40007702019709F071CF8091E800877F809339
:101B5000E8008091E80080FFFCCF80911101809324
:101B6000F1008091E8008E779FCF809172028132E0
:101B700009F05BCF8091760290917702892B69F40E
:101B80008091E800877F8093E8000E949F08809101
:101B90007402809312010E94970C809176029091BA
:101BA0007702019709F041CF8091E800877F809309
:101BB000E8000E949F0880917402809311010E94A6
:101BC000970C33CF80917202813209F02ECF809131
:101BD000E800877F8093E8000E949F08809175024B
:101BE00080933F0322CF80917202813A09F01DCF8A
:101BF0008091E800877F8093E8008091E80080FF73
:101C0000FCCF80913F03ABCF803889F0823849F513
:101C1000809176028F70853020F58093E900809165
:101C2000EB0085FB882780F91092E90006C08091BF
:101C30006F0290917002911182609091E800977FFD
:101C40009093E8008093F1001092F1008091E800F9
:101C50008E7731C0282F2D7F21F48823F1F0823038
:101C600079F18091E80083FF0AC08091E800877FC6
:101C70008093E8008091EB0080628093EB001F70FE
:101C80001093E900AA960FB6F894DEBF0FBECDBF41
:101C9000DF91CF911F910F9108958091740281304F
:101CA00001F7933009F080E0809370021092E90010
:101CB0008091E800877F8093E8000E949F08D1CF41
:101CC000809174028111F2CF809176028F702FEF94
:101CD000280F243030F68093E9002091EB0020FF9C
:101CE000E5CF933031F48091EB0080628093EB007C
:101CF000DDCF9091EB0090619093EB0021E030E01C
:101D000001C0220F8A95EAF72093EA001092EA00B8
:101D10008091EB008860EACF8111A3CF009174021B
:101D20000F778091E3008078802B8093E30080918F
:101D3000E800877F8093E8000E949F088091E80078
:101D400080FFFCCF8091E30080688093E30083E014
:101D5000011101C082E080937A0283CF80588230E3
:101D600008F07FCF20917402309175022C3D83E002
:101D70003807A1F583E08A838AE289834FB7F89414
:101D8000DE01139620E03EE051E2E32FF0E05093B5
:101D90005700E49120FF03C0E295EF703F5FEF70C2
:101DA0008E2F90E0EA30C0F0C7968D939D932F5F01
:101DB000243159F74FBF8091E800877F8093E80076
:101DC0006AE270E0CE0101960E9414088091E8005A
:101DD0008B778093E80045CFC096E7CF809176025D
:101DE00090917702432F55274330510509F44FC096
:101DF00078F54130510509F445C084E590E0E3E110
:101E0000F2E04230510509F02CCF2091E800277F05
:101E10002093E8002091780230917902821793078D
:101E200008F49C0140E02115310509F063C041111F
:101E300061C08091E80082FDC9CF80917A02882339
:101E400029F2853019F28091E80083FFF2CFBECFEE
:101E50004132510509F43FC04232510509F001CF2A
:101E60008330910508F0FDCEFC01EE0FFF1FE35E0D
:101E7000FE4F0190F081E02D865E9E4FDC018C913B
:101E800090E01DC082E190E0E7E6F2E0BECF3327AC
:101E900021303105C1F060F02230310509F0E1CE8A
:101EA000E9E7F2E0E4918E2F90E0E9E7F2E007C085
:101EB000EDEBF2E0E4918E2F90E0EDEBF2E0009795
:101EC00009F4CFCEA2CFEDEAF2E0E4918E2F90E0BC
:101ED000EDEAF2E0F4CF8330910508F0C2CE880F2E
:101EE000991FFC01ED5DFE4F0190F081E02D89E02E
:101EF00090E08BCF80917A02882309F467CF8530F8
:101F000009F464CF8091E80083FD60CF8091E80000
:101F100082FD8FCF8091E80080FF85CF8091F20015
:101F200090E02115310519F08830910550F041E01D
:101F3000089709F040E08091E8008E778093E800F0
:101F400072CF44914093F1003196215031090196AE
:101F5000E8CF803809F085CE8091E800877F8093B4
:101F6000E800809171028093F10070CE811179CEEA
:101F700000917402023008F074CE8091E800877FEF
:101F80008093E800009371020E949F08002399F05B
:101F900084E080937A0242E061EC81E00E94BE0816
:101FA00042E061EC82E00E94BE0846E261EC83E020
:101FB0000E94BE0856CE8091E30087FDE9CF81E004
:101FC000E8CFEF92FF920F931F93CF937C018B0189
:101FD0000E947008C82F811119C08091E80085FD0A
:101FE0000DC08091E8008E778093E8000E94DF0C9E
:101FF0000E947008882389F3C82F08C0F7018191D7
:102000007F018093F1000150110939F78C2FCF9196
:102010001F910F91FF90EF900895882341F08095D4
:1020200090912E03892380932E030C94360C0895EF
:10203000882339F090912E03892B80932E030C94E2
:10204000360C08958732D8F58E3108F0FCC08E30FA
:1020500009F48FC078F4873009F470C08B3009F42C
:1020600056C0863009F458C088E295E00E940D05FC
:1020700080E00895863109F4A6C078F48031A1F794
:1020800090914103892F877F93FF8860809341035C
:1020900083FF7FC082EB96E063C0893109F47CC086
:1020A0008B3111F790914103892F8D7F91FF8260D1
:1020B0008093410381FF5AC08BEE96E051C0883374
:1020C00031F150F4893221F0853311F0873261F615
:1020D00080E00E94BB0C40C08334D1F320F48A33EB
:1020E00018F28953F6CF883409F0BECF0E94970CBE
:1020F00081E197E00E940D052FEF83ED90E32150E1
:1021000080409040E1F700C000000E94F5078EE695
:1021100094E00E940D0520C080914103817F8E7F55
:102120008093410381E095E00E940D0582E297E0F3
:102130000E940D0581E08093400308958091410342
:1021400080FF0CC084E097E00E940D058091410360
:10215000817F8E7F8093410381E0089588EF96E030
:102160000E940D05809141038160F4CF8DED96E0D2
:10217000D0CF90914103892F8B7F92FF8460809311
:10218000410382FF03C08EEC96E0EACF8EEB96E02F
:10219000C0CF85EA96E0BDCF86E996E00E940D05A6
:1021A00081E796E00E940D058AE296E00E940D0507
:1021B00084E096E00E940D058FEB95E00E940D05EE
:1021C00083E995E0A6CF85E895E00E940D050E9481
:1021D000D2071F928F938BE695E09F938F930E9477
:1021E000A605809112011F928F9384E595E09F933D
:1021F0008F930E94A60580913F031F928F9381E4E5
:1022000095E09F938F930E94A6052FB7F894809135
:102210003B0390913C03A0913D03B0913E032FBF3F
:10222000BF93AF939F938F938AE295E09F938F9391
:102230000E94A6058DB79EB742960FB6F8949EBF32
:102240000FBE8DBF89CF8D5144CFCF93DF938823AD
:1022500009F454C09EE7980F933020F5C2E0D9E30B
:10226000823831F0C4E0D7E4833811F4C1E0D3E51B
:102270000E94D2078C2309F441C08D2F0E9476065C
:102280000E94360C2FEF41EE54E021504040504068
:10229000E1F700C000008D2F0E946A06DF91CF9108
:1022A0000C94360C9CEF980F913AB0F390E2980F93
:1022B000983088F4877021E030E0A90102C0440F13
:1022C000551F8A95E2F7CA01809590912E038923C4
:1022D00080932E03E3CF9BE5980F933030F490E08A
:1022E00080E0DF91CF910C94580B885A873130F4FD
:1022F00090E080E0DF91CF910C942C0BDF91CF9197
:102300000895CF93DF93882309F4C2C0C82F8EE7C6
:102310008C0F833030F5C238F1F0C338F9F0C4E0E7
:10232000D7E40E94D2078C2309F0B2C08D2F0E94FF
:1023300076060E94360C2FEF81EE94E0215080400B
:102340009040E1F700C000008D2F0E946A06DF91E7
:10235000CF910C94360CC2E0D9E3E3CFC1E0D3E5D2
:10236000E0CF8CEF8C0F813A08F03FC180914003A1
:102370008130B1F048F0823009F441C0109240033E
:102380008C2F0E947606E3CF809136028E3011F0BA
:102390008730B1F78C2F0E942210811179C0F0CFC5
:1023A000809136028E30B1F38730A1F3C431C9F089
:1023B00048F4CB3059F0C031C1F08FED92E00E946B
:1023C0000D0511C0C93269F0C833B9F781E095E055
:1023D0000E940D0585EE92E00E940D0581E081705E
:1023E000DCCF1092400380E0FACF0E94840B81EE94
:1023F00092E00E940D0582E080934003EFCFC4324B
:10240000D0F4CE3108F0C0C0CB30E9F048F4C7308A
:1024100009F4D1C08EE893E0DF91CF910C940D05C3
:10242000C331C9F1C431B1F780917F02882349F1EA
:1024300010927F020AC0CB3409F4BBC0C0F4C93289
:1024400099F3C83339F70E94840B80917F02882367
:1024500009F4C8C01F928F9388E893E09F938F93ED
:102460000E94A6050F900F900F900F9011C0C135DC
:1024700009F499C0C23509F490C0CE3459F66AE027
:1024800093C08DE993E00E940D0581E080934003A5
:10249000DF91CF91089587E793E00E940D0585E6CF
:1024A00093E00E940D05809118011F928F9382E6A0
:1024B00093E09F938F930E94A60580E693E00E948D
:1024C0000D058EE493E00E940D05809117011F9287
:1024D0008F938BE493E09F938F930E94A60589E4EA
:1024E00093E00E940D058AE393E00E940D05809120
:1024F00016011F928F9387E393E09F938F930E941F
:10250000A60585E393E00E940D0584E293E00E9416
:102510000D05809115011F928F9381E293E09F93A7
:102520008F930E94A6058FE193E00E940D058AE03B
:1025300093E00E940D05809114011F928F9387E014
:1025400093E09F938F930E94A60585E093E00E94FD
:102550000D058EEE92E00E940D05809113011F92F1
:102560008F938BEE92E09F938F930E94A60589EE46
:1025700092E00E940D058DB79EB748960FB6F8946D
:102580009EBF0FBE8DBF61CFCE51EC2FF0E0E75D57
:10259000FE4F808180937F0258CF61E080917F025F
:1025A0000E94880A52CF61E080917F020E94090A4E
:1025B0004CCF6AE0F3CF8EE18093180182E38093E1
:1025C00017018AE08093160184E18093150188E069
:1025D0008093140188E28093130180E993E00E94C4
:1025E0000D0533CF85E893E017CF80E28C0F88305C
:1025F00068F4C77021E030E001C0220FCA95EAF705
:1026000080912E03822B80932E03A1CE8BE58C0F1D
:10261000833070F481E890E0C53A31F083E890E0CF
:10262000C63A11F482E890E0DF91CF910C94580BF8
:1026300088E58C0F873108F02BCF82EE90E0C83A06
:1026400009F460C089EE90E0C93A09F45BC08AEEF3
:1026500090E0CA3A09F456C085EB90E0CB3A09F411
:1026600051C086EB90E0CC3A09F44CC083EB90E08B
:10267000CD3A09F447C084EB90E0CE3A09F442C069
:1026800087EB90E0CF3AF1F18CEC90E0C13BD1F1D7
:102690008DEC90E0C03BB1F183E891E0C23B91F159
:1026A0008AE891E0C33B71F182E991E0C43B51F1CA
:1026B00084E991E0C53B31F181E292E0C63B11F142
:1026C00083E292E0C73BF1F084E292E0C83BD1F0B4
:1026D00085E292E0C93BB1F086E292E0CA3B91F01C
:1026E00087E292E0CB3B71F08AE292E0CC3B51F082
:1026F0008FE690E0CD3B31F090E080E0CE3B11F4EE
:1027000080E790E0DF91CF910C942C0BCF92DF9279
:10271000EF92FF920F931F93CF93DF9300D000D0DF
:102720001F92CDB7DEB76C0185E0F601DE01119690
:1027300001900D928A95E1F7F60140815181238144
:10274000348191E02115310531F05F3F19F491E0BA
:102750004F3F09F090E090FD99C0F6010281F580AD
:10276000F2949FE0F92249835A830B83722F3D83B1
:102770002C83602F8D810E948F06182FE92FE29500
:10278000EF70EF3008F082C0F0E0E753FC4E0C949D
:102790001622D813D813161416148C14BE1446140B
:1027A0004614B0154614861686164614461442176B
:1027B000F92FFF70FF2E907F19F0F29480EFF8222E
:1027C0000023C9F0FF2039F080912D03F82AF09200
:1027D0002D030E94360C812F0F900F900F900F90B9
:1027E0000F90DF91CF911F910F91FF90EF90DF90AD
:1027F000CF900C948111812F0E942511FF2009F4A4
:1028000045C0F09480912D03F822F0922D030F9093
:102810000F900F900F900F90DF91CF911F910F911C
:10282000FF90EF90DF90CF900C94360C892F8F7033
:10283000907F903211F08295807F112379F01130D2
:1028400009F449C0002309F455C0FF2059F0F601EE
:10285000958190FF69C29F70958304C0002321F188
:10286000F1100FC00F900F900F900F900F90DF910D
:10287000CF911F910F91FF90EF90DF90CF900C942C
:10288000181021E0F212EECF80932C030F900F90DE
:102890000F900F900F90DF91CF911F910F91FF90AC
:1028A000EF90DF90CF900895F11011C010922C039B
:1028B0000F900F900F900F900F90DF91CF911F917D
:1028C0000F91FF90EF90DF90CF900C940D1091E05E
:1028D000F912ECCFDBCF002349F0E5E0EF15B0F2C1
:1028E00090912E03982309F4BDCFE2CFF4E0FF15B9
:1028F00068F2DECFFF20E1F2812F0F900F900F9052
:102900000F900F90DF91CF911F910F91FF90EF905B
:10291000DF90CF900C942511892F86958695837032
:10292000C1F0813009F0B2CF812F9370011102C044
:1029300090E080E00F900F900F900F900F90DF913C
:10294000CF911F910F91FF90EF90DF90CF900C945B
:102950002C0B812F9370011102C090E080E00F904A
:102960000F900F900F900F90DF91CF911F910F91CB
:10297000FF90EF90DF90CF900C94580B002309F458
:1029800071C0803FA1F40E94EA05819580933803CD
:102990000F900F900F900F900F90DF91CF911F919C
:1029A0000F91FF90EF90DF90CF900C949B0B813FA5
:1029B00019F40E94EA05EACF823F31F40E94EA0549
:1029C000819580933703E4CF833F19F40E94EA0591
:1029D000F8CF893F29F40E94AF0580933903D8CFFF
:1029E0008A3F21F40E94AF058195F7CF8B3F31F4E8
:1029F0000E94AF05819580933A03CACF8C3F19F4AA
:102A00000E94AF05F8CF809136038160143FA1F09A
:102A1000809136038260153F79F08091360384609F
:102A2000163F51F0809136038860173F29F0183F18
:102A300031F480913603806180933603A9CF809171
:102A4000300381601D3F59F08091300382601E3F4A
:102A500031F01F3F09F09CCF809130038460809358
:102A6000300396CF803FC1F48091380387FD1092E8
:102A700038038091370381118BCF80913803811106
:102A800087CF80913903811183CF80913A038111DF
:102A90007FCF109231037CCF813F29F4809138039E
:102AA00018162CF3E6CF80913703123F29F487FFE5
:102AB000E0CF10923703DDCF133F19F41816CCF393
:102AC000D8CF193F39F480913903181694F6109233
:102AD0003903CFCF1A3F29F48091390387FFC9CF3B
:102AE000F6CF1B3F39F480913A0387FFC2CF109293
:102AF0003A03BFCF1C3F29F480913A031816BCF368
:102B0000B8CF809136038E7F143FA1F080913603B9
:102B10008D7F153F79F0809136038B7F163F51F002
:102B200080913603877F173F29F0183F31F4809159
:102B300036038F7E809336039CCF809130038E7F47
:102B40001D3F59F0809130038D7F1E3F31F01F3FB4
:102B500009F08FCF809130038B7F8093300389CF32
:102B6000892F837009F064C0011190CE812F829566
:102B700086958770880F880F412F4F70C42ED12CF7
:102B8000F12CE12C082E04C0CC0CDD1CEE1CFF1C2B
:102B90000A94D2F740E050E0BA0114FF11C00FE0F0
:102BA00010E020E030E004C0000F111F221F331F8F
:102BB0008A95D2F7B901A801409550956095709516
:102BC0000091420310914303209144033091450347
:102BD0009695969593709230E9F028F5913089F0AA
:102BE0004C295D296E297F294023512362237323B9
:102BF000409342035093430360934403709345030F
:102C000045CEC02AD12AE22AF32A4C295D296E2911
:102C10007F29EECF4C295D296E297F294027512736
:102C200062277327E5CF4023512362237323EDCF1F
:102C30008695002311F0892F8170882309F426CE10
:102C4000812F829586958770880F880F412F4F704E
:102C5000C42ED12CF12CE12C082E04C0CC0CDD1C90
:102C6000EE1CFF1C0A94D2F740E050E0BA0114FFBA
:102C700011C00FE010E020E030E004C0000F111F91
:102C8000221F331F8A95D2F7B901A80140955095AC
:102C9000609570950091B8021091B9022091BA0226
:102CA0003091BB029695969593709230E9F028F595
:102CB000913089F04C295D296E297F2940235123C9
:102CC000622373234093B8025093B9026093BA020F
:102CD0007093BB02DBCD0C291D292E293F29402BE7
:102CE000512B622B732BEECF4C295D296E297F2946
:102CF0004027512762277327E5CF402351236223C2
:102D000073234C295D296E297F29DCCF803F09F48C
:102D10004EC0D0F480E4810F803270F1002309F4BA
:102D2000ACC0FF2009F4A6C0812F0E948111193385
:102D300009F099C0FFEF21EE84E0F150204080407F
:102D4000E1F700C00000A2CD823F09F470C008F492
:102D50005BC0833F19F7002309F47CC0292F2F7132
:102D600081E090E0A0E0B0E004C0880F991FAA1FA6
:102D7000BB1F2A95D2F73AC0E12FE071FE2E892FB2
:102D80008F71002351F00E945C07812F8295807F14
:102D9000F11068CD812F8F7065CD0E943807812F8B
:102DA0008295807FF11084CD812F8F7081CD00239B
:102DB00031F1F4E0FF1508F469CD292F2F7181E07E
:102DC00090E0A0E0B0E004C0880F991FAA1FBB1FCD
:102DD0002A95D2F74091B8025091B9026091BA0297
:102DE0007091BB0284279527A627B7278093B80246
:102DF0009093B902A093BA02B093BB0247CD25E0ED
:102E00002F1508F443CDD9CF892F8F71002399F066
:102E10000F900F900F900F900F90DF91CF911F9117
:102E20000F91FF90EF90DF90CF900C945C07892F6B
:102E30008F71002369F30F900F900F900F900F90F8
:102E4000DF91CF911F910F91FF90EF90DF90CF9086
:102E50000C9438071092B8021092B9021092BA027C
:102E60001092BB0213CD133509F464CF173409F067
:102E70000DCD60CF892F8F71CBCFF1103DCD892F34
:102E80008F71D9CF811102CD002309F4FFCC0E94AC
:102E9000970C8FEF90E7E2E081509040E040E1F73F
:102EA00000C000000E94F5071F93CF93DF9380912D
:102EB0008502807FB1F480918202882391F0209175
:102EC000B70210918602C0918002D0918102A09138
:102ED0008302B091840241E0CF3F09F040E0121339
:102EE00004C0DF91CF911F91089581E0109721F0E8
:102EF000842FDF3F09F080E030E080FD33C0C9015E
:102F000066E070E00E94F121FC01E957FD4F8181EC
:102F10008D1328C080818C1325C08281811122C02D
:102F2000838194818A1B9B0B883C9105D8F4809106
:102F300085028F70806180938502C90166E070E030
:102F40000E94F121FC01E457FD4F90819F70906138
:102F5000908380E892E00E948613DF91CF911F91C9
:102F60000C947C072F5F3F4F2770B9CF9F92AF9291
:102F7000BF92CF92DF92EF92FF920F931F93CF9366
:102F8000DF93CDB7DEB761970FB6F894DEBF0FBE03
:102F9000CDBF8C0185E0F801DE011D9601900D92F8
:102FA0008A95E1F7F80140812181F280C380D480C5
:102FB000909180023091810260918302709184022D
:102FC00081E06115710531F03F3F19F481E09F3FC9
:102FD00009F080E0F82FF1709F2E80FD4EC180E84F
:102FE000A82E82E0B82EE0908202F601E61BF70BD5
:102FF000EE2009F404C180918502582F507FE83CEF
:10300000F10508F0BDC0511183C0EF2C321322C06E
:10301000941320C0F1101EC08F70806180938502D0
:10302000C5010E94861380918502F80185838E2D4B
:1030300061960FB6F894DEBF0FBECDBFDF91CF9182
:103040001F910F91FF90EF90DF90CF90BF90AF90C6
:103050009F90089581E0C114D10431F02F3F19F4FD
:1030600081E04F3F09F080E080FD14C081E08F25B2
:10307000F82FF170BF2EE091B7023091860280FDEB
:1030800022C0FF20A1F28091850281608093850299
:10309000E12CCDCF80E0ECCFF0E0CF0166E070E036
:1030A0000E94F121DC01A957BD4F11968C91119717
:1030B000281307C08C91481304C012968C918F116D
:1030C000E0CF3196E770E313E7CF7C2DD98AC88A29
:1030D000522F6F2D89890E948F06292F22952F70DC
:1030E000223050F0243078F49F7051F0F80195812F
:1030F000907F31F4E92C9BCF9F7011F08823D1F39E
:10310000805E8830B8F3C8010E9486139B2CF2CFF2
:10311000321306C0941304C0F801FF2009F48AC0DA
:103120004D872E87FF867C2DD98AC88A522F6F2D16
:1031300089890E948607882309F4AEC0FF2009F41C
:10314000ABC080918502803270F020918002309176
:10315000810238872F831986DB86CA868C87CE0149
:1031600007960E94861386E0F801A0E8B2E001907D
:103170000D928A95E1F70E945417EE24E39457CFFD
:1031800051110AC080E892E00E94861386E0F501A2
:1031900011928A95E9F77CCF32130FC094130DC0BA
:1031A000F1100BC0F8018583C8010E94861386E0E8
:1031B000F50111928A95E9F73ACF4D872E87FF8660
:1031C0007C2DD98AC88A522F6F2D89890E94860743
:1031D000882309F461C0FF2009F45EC08091850254
:1031E000803208F220918002309181023A83298353
:1031F0001B82DD82CC828E83CE010196B2CFE83C69
:10320000F105A8F6EF2CFF2009F446C032131FC0C9
:1032100094131DC08091850280FD10C0982F907F6F
:1032200069F0F8018583903F31F0982F907F905F8F
:103230008F70892B8583C8010E94861386E0F80170
:10324000A0E8B2E001900D928A95E1F7F0CE4D87AB
:103250002E87FF867C2DD98AC88A522F6F2D8989A7
:103260000E94860781117FCF8091850281608093C3
:103270008502C8010E948613DACEFF2069F04D87CF
:103280002E87FF867C2DD98AC88A522F6F2D898977
:103290000E948607811167CFC8010E9486136DCFF7
:1032A000CF93DF93CDB7DEB767970FB6F894DEBF45
:1032B0000FBECDBF4B8B5C8B6D8B7E8B8F8B1A8A39
:1032C000198A85E0FE017396DE011D9601900D922C
:1032D0008A95E1F786E0FE013D96DE0117960190A2
:1032E0000D928A95E1F7CE0107960E94B6178111DB
:1032F00038C086E0FE013796DE01119601900D92EE
:103300008A95E1F79F8188852A853B85232B39F0B3
:103310008F3F19F481E09F3F19F080E001C081E008
:1033200080FD1FC08091860290E09C012F5F3F4F7F
:10333000277033274091B7024217130661F166E008
:1033400070E00E94F121DC01A957BD4F96E0FE011B
:10335000319601900D929A95E1F7209386020E9492
:103360007C078091B70290918602891709F190E05D
:1033700066E070E00E94F12189579D4F0E94B617C8
:103380008823B1F08091B70290E001968770992769
:103390008093B702E6CF0E94970C1092860210929B
:1033A000B70286E0E0E8F2E0DF011D928A95E9F7D6
:1033B00067960FB6F894DEBF0FBECDBFDF91CF91F9
:1033C0000895CF93DF9300D01F92CDB7DEB7209141
:1033D0007A02243021F523E029839B838A8382E0CB
:1033E0008093E9008FEF9091E800815095FD06C031
:1033F00095ED9A95F1F700008111F5CF8091E800E5
:1034000085FF0DC050E040E063E070E0CE01019622
:103410000E94E10F8091E8008E778093E8000F9082
:103420000F900F90DF91CF910895CF93DF9300D04D
:103430001F92CDB7DEB720917A02243061F5198250
:103440001A821B8222E029838138910520F080585E
:1034500091099B838A8382E08093E9008FEF9091AA
:10346000E800815095FD06C095ED9A95F1F70000B2
:103470008111F5CF8091E80085FF0DC050E040E05C
:1034800063E070E0CE0101960E94E10F8091E800B8
:103490008E778093E8000F900F900F90DF91CF917F
:1034A000089520917A02243049F522E02093E90022
:1034B0002FEF3091E800215035FD06C035ED3A95EB
:1034C000F1F700002111F5CF2091E80025FF16C08B
:1034D0002091110150E040E063E070E0222339F0D8
:1034E00021E02093F10050E040E065E070E00E94B0
:1034F000E10F8091E8008E778093E8000895CF93E4
:10350000DF9320917A02243011F521E02093E90025
:1035100021E8215021F03091E80035FF1BC02091B7
:10352000E80025FF14C0EC0150E040E068E070E0E6
:103530000E94E10F8091E8008E778093E80088E098
:10354000FE01A7E6B2E001900D928A95E1F7DF91C6
:10355000CF910895EFE3F1E03197F1F700C000005B
:10356000D8CF5198599A85E08A95F1F7000089B132
:10357000869581700895CF93DF93EC010E94B11A74
:10358000882311F0209721F4CE01DF91CF91089587
:1035900085E08A95F1F700002197F0CF0F931F93F4
:1035A000CF93DF9310924102CAEFD0E088EE93E010
:1035B0000E94BB1A892B21F42197C1F781E00AC030
:1035C000D8E0C0E0CC0F88EC90E00E94BB1A892BB9
:1035D000B9F582E0809341028FE991E00E940D05E8
:1035E000809141021F928F938AE991E09F938F937C
:1035F0000E94A60588E991E00E940D059FEF29E64B
:1036000088E1915020408040E1F700C000000E9416
:10361000FA090E94F4090F900F900F900F90CFEFCE
:1036200023C025E02A95F1F70000015011090E94FE
:10363000B11A811108C00115110599F783E0CACFAD
:1036400008EC10E0F4CF012BC9F35098589A85E0AC
:103650008A95F1F700004899C160D15009F0B2CFC6
:103660000E94FA090E94F4098C2FDF91CF911F91DB
:103670000F910895EF92FF920F931F93CF93DF93D3
:10368000E82E109241020E94FA090E94F709CAEF3F
:10369000D0E088EE93E00E94BB1A892B21F4219799
:1036A000C1F781E00BC008E010E080E8F82E8AEF57
:1036B00090E00E94BB1A892B41F583E08093410280
:1036C00087E891E00E940D05809141021F928F933F
:1036D00082E891E09F938F930E94A60580E891E095
:1036E0000E940D059FEF29E688E19150204080401F
:1036F000E1F700C000000E94FA090E94F4090F904F
:103700000F900F900F9080E02AC08E2D8F2161F0D6
:103710000E94F409C8ECD0E00E94B11A81110DC0DA
:10372000209729F484E0CACF0E94F709F3CF25E05F
:103730002A95F1F700002197EFCFCD2B99F3F6945E
:103740000150110909F0B3CF8FE891E00197F1F72B
:1037500000C000000E94FA090E94F40981E0DF9194
:10376000CF911F910F91FF90EF900895CF9384E137
:103770000E943A1B0E94CE1AC82F8B37C1F080914D
:10378000410380FF0CC01F92CF9382EB91E09F9387
:103790008F930E94A6050F900F900F900F9080912D
:1037A000410380FF04C080EB91E00E940D058C2F47
:1037B000CF9108951F93CF93DF93809100018F3FA6
:1037C000D1F486E10E943A1B0E94CE1A8093000138
:1037D0008F3F29F480E0DF91CF911F9108951F92D0
:1037E0008F9383E791E09F938F930E94A6050F909C
:1037F0000F900F900F90C0914002CC2351F0109287
:103800004002CB3739F3CF3F09F08BC0C0930001A2
:10381000E1CFC0913F02CC2319F010923F02F1CFCB
:10382000C0913E02CC23E1F010923E028C2F8F77A4
:10383000813721F1893779F50E94B61BC82F8F7720
:103840008D3019F088F4853099F48C2F0E94FD0991
:10385000C7FF0EC0C82FC064806680934002D1CFDE
:103860000E94B61BC82FE2CF813179F38B3169F307
:103870008C2F0E94FD09C82FC064C3CF0E94B61BC5
:10388000982F9F77913729F0993751F00E94FD09C1
:1038900030C080933E028C2F0E94FD09C82FB1CF0B
:1038A0000E94B61BD82F8F778D3019F0D0F4853059
:1038B000E1F4C7FF21C08C2F0E94FD09C82F8FE5BE
:1038C00091E0D7FF2BC084E691E00E940D05C093E4
:1038D0003F028D2F0E94FD09982F90669093400221
:1038E000CACF813131F38B3121F38D2F0E94FD0935
:1038F000806480934002CFCF8D2F0E94FD09182F46
:10390000C82FC06685E591E0D7FF08C08AE591E041
:103910000E940D05C0934002C12FAECF0E940D053D
:1039200070CF2091510230915202EC2FE695E6952E
:10393000E6954C2F477081E090E001C0880F4A95D2
:10394000EAF7C7FF22C0EF70E20FF32FF11D809559
:103950009081892380838091410380FF14C081E797
:1039600091E00E940D051F92CF938CE691E09F930A
:103970008F930E94A60589E691E00E940D050F90A5
:103980000F900F900F9081E026CFE20FF32FF11DE3
:103990009081892BDFCF78941F920F920FB60F92F0
:1039A00011248F939F93AF93BF9380913B0390918A
:1039B0003C03A0913D03B0913E030196A11DB11DB2
:1039C00080933B0390933C03A0933D03B0933E034D
:1039D000BF91AF919F918F910F900FBE0F901F904D
:1039E00018951F920F920FB60F9211248F939F93E9
:1039F000AF93BF9380912F03811113C080913B033C
:103A000090913C03A0913D03B0913E034196A11DCE
:103A1000B11D80933B0390933C03A0933D03B0936F
:103A20003E03BF91AF919F918F910F900FBE0F906A
:103A30001F9018951F920F920FB60F9211242F937B
:103A40003F934F935F936F937F938F939F93AF9326
:103A5000BF93EF93FF938091E10082FF09C08091B3
:103A6000E20082FF05C08091E1008B7F8093E1003E
:103A70008091E10080FF1FC08091E20080FF1BC0A9
:103A80008091E2008E7F8093E2008091E20080616D
:103A90008093E2008091D80080628093D80019BCA6
:103AA00085E080937A02809166028093650210928D
:103AB00066020E94970C8091E10084FF2DC08091E6
:103AC000E20084FF29C084E089BD86E089BD09B495
:103AD00000FEFDCF8091D8008F7D8093D80080912B
:103AE000E1008F7E8093E1008091E2008F7E8093E1
:103AF000E2008091E20081608093E2008091710297
:103B0000882309F440C084E080937A020E94970CD5
:103B100080916502809366028091E10083FF22C05C
:103B20008091E20083FF1EC08091E100877F809337
:103B3000E10082E080937A02109271028091E100AC
:103B40008E7F8093E1008091E2008E7F8093E2007F
:103B50008091E20080618093E20042E060E080E0DA
:103B60000E94BE08FF91EF91BF91AF919F918F91FD
:103B70007F916F915F914F913F912F910F900FBE69
:103B80000F901F9018958091E30087FD02C081E09F
:103B9000BBCF83E0B9CFCF93DF93CDB7DEB72B9701
:103BA0000FB6F894DEBF0FBECDBF84B7877F84BF4A
:103BB0000FB6F894A89580916000886180936000AA
:103BC000109260000FBE80E890E00FB6F8948093EA
:103BD0006100909361000FBE8BE099E090933501F6
:103BE0008093340187E091E0909333038093320314
:103BF0008AEF91E00E940D050E94DE07809163002C
:103C00008E7F8093630081E0809364021092E200D3
:103C10001092E1008091D8008F778093D800809136
:103C2000D80080688093D8008091D8008F7D8093E1
:103C3000D80084E089BD86E089BD09B400FEFDCFCF
:103C400010927A02109271021092700210926F021A
:103C500042E060E080E00E94BE088091E1008E7F3B
:103C60008093E1008091E20081608093E200809186
:103C7000E20088608093E2008091E0008E7F809374
:103C8000E000789482E084BD93E095BD9AEF97BD03
:103C900080936E00809141038160809341030E9474
:103CA000FA090E94F4092FEF83ED90E32150804040
:103CB0009040E1F700C00000E3E4F2E081E592E02B
:103CC00011928E179F07E1F783E492E090935202DE
:103CD00080935102569A5E9AEFEFF9E628E1E1509F
:103CE000F0402040E1F700C00000569A5E988091B5
:103CF0007A02843009F037C10E94F308882309F45E
:103D000032C188EE91E00E940D058AED91E00E949B
:103D10000D05F9E14F2EF1E05F2EA7EB6A2EA1E031
:103D20007A2EBFECAB2EB1E0BB2E18E1812E912C88
:103D300080917A02853009F419C10E94DA1BE4E50A
:103D4000CE2EE2E0DE2EF12CE12CEB86E09151024A
:103D5000F0915202EE0DFF1D3080F60120802314F9
:103D600009F45FC08091410381FF38C082EC91E08B
:103D70000E940D0510E000E0E0915102F091520226
:103D8000E00FF11F2081229530E0C901880F991FB3
:103D9000880F991F8C7C359527953595279523732A
:103DA000822B90E05F924F929C01220F331F2A7A60
:103DB000959587958575822B1F928F931F930F93EF
:103DC0007F926F920E94A6050F5F1F4F0FB6F89467
:103DD000DEBF0FBECDBF0E30110571F600E011E061
:103DE0002324822D8123C9F00E839B859F8391E03C
:103DF000812F832109F490E098870E945E068160FC
:103E0000782F9A8789874E815F8168858A850E948D
:103E10005019F6018081812780830F5F110F0830D0
:103E200001F7FFEFEF1AFF0A2FEFC21AD20A8EE056
:103E3000E816F10409F089CF9FEF99839A831B82DA
:103E40000E945E068160782F9D838C8349815A8110
:103E50006B818D810E9450198091340390913503BC
:103E60002FB7F89440913B0350913C0360913D0380
:103E700070913E032FBFFA01E81BF90B209131032B
:103E80008091170190E0211107C08091180190E006
:103E90006AE070E00E94F121E817F90780F0809154
:103EA0003703F09038031091390300913A038111E0
:103EB00097C0F11059C1111157C1011155C10E948C
:103EC000D207909153028917C9F00E94D2078093BC
:103ED0005302909141039570953051F41F928F9346
:103EE000BF92AF920E94A6050F900F900F900F9077
:103EF00080915302569A81FFE1C05E9A2091E400BE
:103F00003091E50080916202909163022817390791
:103F100039F18091E4009091E500909363028093E1
:103F200062020E94F3088823D9F080917A028430DB
:103F3000B9F48091E9008F709091EC0090FFC0C0BF
:103F400090E8892B93E09093E9009091EB0090FF2B
:103F500004C09091EE0097FDD1C08F708093E9006E
:103F60000E94DF0CE5CE0E94DF0CC1CE80917A0268
:103F7000843011F110922F0380E40FB6F894A895C5
:103F8000809260000FBE8093600083B7817F846061
:103F900083BF83B7816083BF7894889583B78E7F12
:103FA00083BF0FB6F894A8958091600088618093D4
:103FB0006000109260000FBE80917002882309F4A7
:103FC000B7CE0E94DA1BE0915102F0915202CF016C
:103FD0000E9621912111B2C08E179F07D1F7A8CE5E
:103FE0002F3F19F02F5F20933103181624F40E94FD
:103FF000EA05809337038091370387FF05C00E944D
:10400000EA058195809337031F1424F40E94EA0582
:10401000809338038091380387FF05C00E94EA052A
:1040200081958093380360913703662331F1F090D6
:104030003803FF2011F1062E000C770B880B990B2B
:104040000E94F02023E333E343E35FE30E94542123
:104050000E94B820609337036F2DFF0C770B880BFD
:10406000990B0E94F02023E333E343E35FE30E94D4
:1040700054210E94B82060933803111624F40E9442
:10408000AF05809339038091390387FF05C00E94F3
:10409000AF05819580933903101624F40E94AF0573
:1040A00080933A0380913A0387FF05C00E94AF05D1
:1040B000819580933A030E949B0B01CF5E981ECF9F
:1040C00090E03FCFE0910201F0910301E90FF11D73
:1040D00020819F5F309106019323909305012093E7
:1040E000F1009091E80095FD09C09091E80090FFE3
:1040F00005C09091E8009E779093E80090910501AB
:1041000020910401291721F02091E80025FDDACF44
:104110009091F200992309F420CF9091E80090FF4C
:104120001CCF9091E80095FD06C09091E8009E7725
:104130009093E80012CF1092F100F3CF84E089BD94
:1041400086E089BD09B400FEFDCF8091D8008F7D47
:104150008093D8008091E00082608093E00080919D
:10416000E00081FDFCCFE4CD2F3F09F03BCF4CCFE9
:104170000E94BF206894B1110C944E2108950E94B2
:10418000332188F09F5798F0B92F9927B751B0F095
:10419000E1F0660F771F881F991F1AF0BA95C9F7CB
:1041A00014C0B13091F00E944D21B1E008950C94FB
:1041B0004D21672F782F8827B85F39F0B93FCCF3AE
:1041C000869577956795B395D9F73EF49095809548
:1041D000709561957F4F8F4F9F4F0895E89409C068
:1041E00097FB3EF490958095709561957F4F8F4F2A
:1041F0009F4F9923A9F0F92F96E9BB279395F69540
:10420000879577956795B795F111F8CFFAF4BB0FBD
:1042100011F460FF1BC06F5F7F4F8F4F9F4F16C021
:10422000882311F096E911C0772321F09EE8872FAB
:10423000762F05C0662371F096E8862F70E060E067
:104240002AF09A95660F771F881FDAF7880F9695E0
:10425000879597F9089557FD9058440F551F59F0C9
:104260005F3F71F04795880F97FB991F61F09F3F63
:1042700079F087950895121613061406551FF2CF8C
:104280004695F1DF08C0161617061806991FF1CFDC
:1042900086957105610508940895E894BB27662703
:1042A0007727CB0197F908950E9466210C94E021AD
:1042B0000E94D22138F00E94D92120F0952311F0DC
:1042C0000C94C9210C94CF210C944E210E942B21D7
:1042D00078F39923C9F35523B9F3950F50E0551F8F
:1042E000AA27EE27FF27BB2700240894679520F410
:1042F000E20FF31FB41F0A1E220F331F441FAA1F11
:104300006695A9F7779530F4F30FB41F0A1E121EB5
:1043100008F46395330F441FAA1F221F769599F75F
:10432000879520F4B40F0A1E121E631F440FAA1FA4
:10433000221F331F8695A9F7862F712D602D11241A
:104340009F5750409AF0F1F088234AF0EE0FFF1F7C
:10435000BB1F661F771F881F91505040A9F79E3FD3
:10436000510580F00C94C9210C944E215F3FE4F379
:10437000983ED4F3869577956795B795F795E79529
:104380009F5FC1F7FE2B880F911D9695879597F932
:10439000089597F99F6780E870E060E008959FEFC7
:1043A00080EC089500240A941616170618060906CC
:1043B000089500240A94121613061406050608959B
:1043C000092E0394000C11F4882352F0BB0F40F423
:1043D000BF2B11F460FF04C06F5F7F4F8F4F9F4F63
:1043E00008950024552704C0080E591F880F991FEF
:1043F000009729F076956795B8F37105B9F7802D88
:10440000952F089597FB072E16F4009407D077FD9B
:1044100009D00E941C2207FC05D03EF4909581959E
:104420009F4F0895709561957F4F0895EE0FFF1F80
:104430000590F491E02D0994AA1BBB1B51E107C024
:10444000AA1FBB1FA617B70710F0A61BB70B881F24
:10445000991F5A95A9F780959095BC01CD010895B3
:04446000F894FFCFFE
:10446400FF0536010000FFF0087F1A511A151AE102
:104474001901012808140A321E00407F22150196F2
:1044840000740025023E02570201020304050607D8
:044494000809000013
:106800000000000000000000040005000600070072
:10681000080009000A000B000C000D000E000F001C
:1068200010001100120013001400150016001700CC
:10683000180019001A001B001C001D001E001F007C
:10684000200021002200230024002500260027002C
:10685000280000002A002B002C002D002E002F0005
:10686000300031A1320033003400350036003700EB
:106870003800E00000000000000000000000000000
:106880000000000000000000000000000000000008
:1068900000000000000000000000000000004F00A9
:1068A000500051005200530067005400550056003C
:1068B000580059005A005B005C005D005E005F00FC
:1068C0006000610062006300640000005700000087
:1068D00000000000000000000000000000000000B8
:1068E00000000000000000000000000000000000A8
:1068F0000000E100E200E300000000000000F1A160
:106900000100010001000100EA4401000100E2442D
:106910000100010001000100460001004A004B0097
:10692000010001004700480001000100E9440100A6
:106930000100010001000100010001003A003B00DC
:106940003C003D003E003F0040004100420043004B
:10695000010000004C00010001004400450052000D
:1069600049000100010050004F0029004D004E0079
:1069700051000100010001000100010001000100BF
:1069800001000100010001000100010001000100FF
:1069900001000100010001000100010001004D00A3
:1069A0004A004E004B0001000100010001000100FF
:1069B00001000100010001000100010001000100CF
:1069C00001000100010001000100010001000100BF
:1069D00001000100010001000100010001000100AF
:1069E000010001000100010001000100010001009F
:1069F000010001000100010001000100010001008F
:00000001FF
